:020000020000FC
:1000000027C018E01A95F1F708950AE03095089492
:1000100010F4C29A02C0C2980000F3DFF2DF3695F6
:100020000A95B1F7089509E0B19BFECFEADFE9DF59
:10003000E8DF8894B19B08940A9511F04795F7CFB3
:1000400008951FEF2AE02A95F1F71A95D9F7089538
:1000500010E820E016BD26BD11E01EBF1FE51DBF44
:10006000C29ABA9AC198B9983C9A3F9A3E983B98DE
:100070003A9A399A389A3D9A379A3598329A3198FD
:10008000309A1AE223E3277F12601160106810642F
:100090001F7D1F7E2B7F2D7F21601ABD23BFB89A45
:0E00A00030E0369AB2DF3699FECF35B1FACF96
:00000001FF
